:030000000219FDE5
:03000B000200AA46
:03002B000201656A
:03005B000202F8A6
:030073000202DEA8
:1000800002030406080C10182030406080040608A3
:100090000C10182030406080A0C000070F1F3F0DDB
:1000A0000D04050D050305030302C2AFC0D0C0E077
:1000B000206217E5256002E473E525F4F58A758B67
:1000C00000D262D0E0D0D0D2AF3285268AC262E5BB
:1000D00026F46035306803207210758B00D0E0D0B4
:1000E000D0C2B1C287C281D2AF32C2B1C287C2818F
:1000F000206E0C206609740AD5E0FDE57E4280750D
:100100008B00D0E0D0D0D2AF32758A00C28DD262DF
:1001100001FF01B9306805206602D2B101B930682B
:1001200005206602D28701B9306805206602D281B7
:1001300001B9C28230680A2066077408D5E0FDD292
:10014000B101B9C28630680A2066077408D5E0FD9F
:10015000D28701B9C28030680A2066077408D5E0EA
:10016000FDD28101B9C2AFC2AD53E6EFC0D0C0E04D
:10017000D2D3D2AFC2CEE52A6007207449152A2116
:10018000C67800790020742EE580307E01F430E5D9
:100190000278FF53DACF207E0343DA20307E034318
:1001A000DA10C2D8C271E580307E01F430E5027900
:1001B000FFC3E89970CB306103752A18207403756A
:1001C0002A18885FD27020740DE52B6004152B214E
:1001D000D643DA01C2D82070024134A85F20610200
:1001E000C2702074367982B70431C3E894F04003BA
:1001F00074F0F8E8C4540F28F87984B70302411B5F
:10020000C313C3138721200802C313200A06C3C8DF
:1002100098F8411B28F8500374FFF88822E52D5404
:10022000066011E533C313C31324062522F52250BB
:10023000037522FF7882B60459852224A824C3E5D9
:100240002495644002A864C3E895664002A86688C5
:1002500025E56970024185C3E8AA699A5003E8FA66
:10026000E4F9EAC333FBE56BF45B29400D256AF83A
:10027000E56A6002156A400B41850AC3E56A9A5037
:1002800002056A78FF8826C26EC3E52694F840020C
:10029000D26EC3E52594404002D26420CF0AD0E05C
:1002A000D0D043E610D2AD32C2CF053A7801E52A6C
:1002B0006005307402152AC3E55F9401400575623C
:1002C0000041D4756300756C00E5622401F562504D
:1002D000037562FFD0E0D0D043E610D2AD32C2AF9A
:1002E000C0D053E67FC260759100855694855795BE
:1002F000759104D0D0D2AF32C2AF53E6EFC2ADC0D9
:10030000D0C0E0C0F0D2D3D2AFA8FBA9FCC2D83095
:100310007102615F53DACF207E0343DA10307E032F
:1003200043DA20D271E580307E01F420E5026136A7
:1003300088278928A18653DACF207E0343DA20302C
:100340007E0343DA10C2D8C271307402A172780001
:10035000E580307E01F430E502A172885FA15A5336
:10036000DACF207E0343DA20307E0343DA10C271F5
:10037000206102813853DACF207E0343DA10307EC9
:100380000343DA20C2D8D271885A895BC3E89558F2
:10039000F8E99559F97B007E087A00C3E8948CE966
:1003A00094005005755E00812A882178A2E6A82174
:1003B0006055C3E894C8E994005008E4D2E4FB7A9D
:1003C0000A8105C3E89468E994015008E4D2E3FB8C
:1003D0007A0F8105C3E894D0E994025008E4D2E290
:1003E000FB7A1E8105C3E894A0E994055008E4D285
:1003F000E1FB7A3C8105C3E89498E994085008E44D
:10040000D2E0FB7A787E00C3E8955CFCE9955DFD5F
:1004100030E70AECF42401FCEDF43400FD755E00D5
:10042000C3EC9AED9E5003755E01885C895D855A28
:1004300058855B597802A15AC3E89527F8E99528B1
:10044000F9307C02A13E307B02A13E307A02A13716
:10045000207502815BE9FDE8FC817AE9C313F9E8C4
:1004600013F8307902A137E9C313F9E813F83078AB
:0F04700002A137E9C313FDE813FC206126C3EC9A
:10047F00941CED940240028191ED7018C3EC94C866
:10048F0050120529C3E529940A5002A172755F0025
:10049F00D270A172E529600215297888E6F97400F7
:1004AF00207F087896B90302789EE624FAFEE4349A
:1004BF0000FFC3EC9EFCED9FFD9208B90310A2084C
:1004CF005007207609D27681DD307602C276A208F7
:1004DF005016B9030DECF42401FCEDF43400FD02C9
:1004EF0004F778007900A13EB90315EC33FCED3326
:1004FF00FDC3EC940AFCED9400FD50047C007D00DC
:10050F00C3EC94FFED9400400678FF7900A13EEC18
:10051F008575F0A4C5F0A2F733F879004003020502
:10052F005A78FF790002055AE9C313F9E813F83036
:10053F007C0EE9600278FFC3E81338F8E43400F961
:10054F00C3E894FFE99400400278FF885FD27020DF
:10055F006102A172741FF4552F4BF52FC274EB700B
:10056F0002D274752A18307403752A0A306102A1F9
:10057F008620740353DAFE207403752B06D0F0D057
:10058F00E0D0D0D2AD43E6103279010205B679033F
:10059F000205B6790A0205B6791E0205B67964021C
:1005AF0005B679C80205B67817E4D5E0FDD8FAD9B3
:1005BF00F6227A147B780205DD7A107B8C0205DD3A
:1005CF007A0D7BB40205DD7A0B7BC80205DD79025B
:1005DF00B27DE4C286D5E0FDD287D5E0FDC287D5D6
:1005EF00E0FDD286D5E0FDD2B1E576D5E0FDC2B112
:1005FF007496D5E0FDD9D9EAF8D5E0FDD8FBDBCE6E
:10060F00C28622C37C007D0075F00005F0EA33FA44
:10061F00EB33FB50F6EB13FBEA13FAC3E9FFE8FEEB
:10062F00E89AF8E99BF95004EFF9EEF8B3EC33FCD4
:10063F00ED33FDD5F0DFEDF9ECF822E889F08A20F3
:10064F00D2D4F8A9F07B0030F70B7BFFF42401F82C
:10065F00E9F43400F9E88520F0A4ADF0F8E985203D
:10066F00F0A4AFF0FEED2EF974003FFA7C04C3EA5C
:10067F0013FAE913F9E813F8DCF48BF030F70AE812
:10068F00F42401F8E9F43400F9E889F0C2D4F8A9A8
:10069F00F0227882B604030206FCC3E55F940140A2
:1006AF00030206C6852224E4F545F546F547F548CD
:1006BF00F549C26D0206FC7882E6FCD26DE522F5A3
:1006CF0023783879C7AA40AB41C3EB13FBEA13FA7F
:1006DF00EC146013C3EB13FBEA13FAEC141460076A
:1006EF00C3EB13FBEA13FAD1128845894622C3E5FF
:1006FF00459523F8E5469400F9500CC3E89480E93A
:10070F0094FF401602072DC3E8947FE9940050032D
:10071F0002072D787F790002072D788079FF884AAC
:10072F00894B22E54A2547F8E54B3548F9854B209B
:10073F00E4300701F43549FA30E709C3EA94F04091
:10074F001502076BC3EA940F500302076B78FF790A
:10075F00FF7A0F02076B780079007AF0C3E52495D2
:10076F0064500AC374019524500B020789E54B208E
:10077F00E70E020789E54B30E706884789488A4923
:10078F002278A4E6FAC3E54A33F8E54B33F9D14AA8
:10079F00E930E70BC3E89480E994FF4013E1C3C34A
:1007AF00E8947FE994005002E1C3787F7900E1C3B8
:1007BF00788079FFE820E715C3E52398F84009C34F
:1007CF00E8940140030207EA78010207EAE8F424FB
:1007DF00012523F840030207EA78FF884C2278A509
:1007EF00E6FAA848A949D14AE930E70CC3E89401D1
:1007FF00E994FF401602081EC3E894FFE9940050E5
:10080F000302081E78FF790002081E780179FFE9BC
:10081F0020E715C3E54C98F84009C3E8940140035D
:10082F000208457801020845E8F42401254CF840F8
:10083F000302084578FF88242278FFC26420693DAF
:10084F00206A12D264C3E541940A4009C3E5259496
:10085F00405002C26479A1E76023E541601F74FF35
:0F086F008541F0848539F0306A0375F005A4F8EF
:10087E00C5F0600278FFC3E895675002A8678866E6
:10088E0022C3E5409440E5419401E566500314010E
:10089E00A0046002F566220208A82275E89022786C
:1008AE0083E6FFE5E820ECF7A8BDA9BE0573C3E516
:1008BE007394084052757300E9FA79A0E76044EA30
:1008CE007007E574601B0208E3C3E895746010E5D9
:1008DE00745006600C140208EF0460F90208EFE58C
:1008EE0074F574C394A8401B7564C0C3940540137B
:1008FE00756480C39405400B756440C39405400332
:10090E0075640075BB0622E5642410500274FFF571
:10091E00647982B70402213CC3A864E5249850028E
:10092E00A824C3E895664002A86688258826E57344
:10093E00B4070375BB1E22743279A687F0A4C5F0E6
:10094E00A2F733F8C3E895644002A864882288248D
:10095E00882588268867227540007541F022C2AF2F
:10096E0075C820A8CCA9CDAA3A30CF010A75C824E3
:10097E00D2AFAB3BAC3C883B893CC3E89BF8E99CCF
:10098E00206908F9306702418121DEAD3D8A3DF9CB
:10099E00EA9DFA600478FF79FFAE3EAF3F8B3E8C46
:1009AE003FC3EC9FFCC3E99CF542A83BA93CC3E8BE
:1009BE009EF8E99FF9C3E54113FBE54013FAE82AD7
:1009CE00F540E93BF54150067540FF7541FF412862
:1009DE00AA40AB41AC40AD417E047F02C3EB940410
:1009EE0040021E1FC3EB940840021E1FC3ED13FDF1
:1009FE00EC13FCDEF7C3EA9CFAEB9DFBEF6009C338
:100A0E00E913F9E813F8DFF7EA28FAEB39FB8A4025
:100A1E008B4150067BFF8B408B41C3EB94025002FF
:100A2E00D2673069047F0341537892E6FFC3E537FE
:100A3E00948240110FC3E53794A040010FC3EF9489
:100A4E000640027F057E05E541C4540FF9E541C419
:100A5E0054F0F8E540C4540F28F8C3E89EFAE99420
:100A6E0000FB4009C3EA9402EB940050047A02E4BE
:100A7E00FB41CDAA40AB41EBC4FEEAC4540F4EFC81
:100A8E00C3EA9CFAEB9400FBC3E813C313F8EA28FD
:100A9E00FAEB3400FB8A408B41C3EB94024002C256
:100AAE00677805EBC4FE7B00EAC4540F4EFAC3EA26
:100ABE0098FA4005C3940250027A027892E6FF300B
:100ACE00600241CD855256855357D26043E680C3AE
:100ADE00E49AF8E49BF93067026167E8FAE9FBD320
:100AEE00E913FDE813FC88528953C3EF9403603871
:100AFE00EF20E00DE82CF8E93DF9ECFAEDFB020BE6
:100B0E0022E828F8E939F9C3E82402F8E93400F9B3
:100B1E007AFE7BFFC3EF9403400E8A548B55884EAA
:100B2E00894F8C508D51619B885489558A4E8B4FBD
:100B3E008C508D51306920C3E53394034019E54242
:100B4E00A2E713F8E555F4240138400B20E70875A9
:100B5E0054FFF42401F555619BE8FAD3E813FC88A1
:100B6E0052C3EF94036020EF20E007E82CF8ECFA74
:100B7E006187E8282402F87AFEC3EF940340088ABE
:100B8E0054884E8C50619B88548A4E8C50E56BC3B2
:100B9E00335002646BF56B30600261A5753402D27E
:100BAE006043E680E52D54066026A840A941C3E9BE
:100BBE0013F9E813F8C2AF53E67F759100C3E498BA
:100BCE00F594E499F595759104D26043E680D2AF21
:100BDE0022D265754400752000306B0375204002EB
:100BEE000BFED265754400752040306B03752000F6
:100BFE00D2AF7801206722E52D54066002C265C38C
:100C0E00E541940540137802940540087803940555
:100C1E0040027806306902780A206019E5446015B2
:100C2E0030690AC3E53394034003D53406D2AFD2FC
:100C3E006C81CF71ADD2AF0000C2AF206726E54107
:100C4E00C3FB940F40027B0FEB240530730123305E
:100C5E006A02742820620123F93069027982E58BD9
:0F0C6E00C39940B50544E59B5440B5200281B9B8
:100C7D0030690A08C3E8940A4001088127206502FB
:100C8D0061FEC26553E67F75910030671075940063
:100C9D007595FE759104D26043E68061FEAE40AF5E
:100CAD0041C3E49EF594E49FF59581A0C3E533948B
:100CBD0002500261FE30650261FED80281CD8127AE
:100CCD00C26C53E67F759100855494855595759149
:100CDD0004854E56854F57D26043E680D2AFE52D41
:100CED0054066008206A020533020D09306C0D2090
:100CFD006B0A2065071581158102158F227800304A
:100D0D0064053065027801E53775F007A4F9E5F063
:100D1D0028F5F0E9A2F013A2F113A2F213F537C3EF
:100D2D0094785003753778C3E53795384008D26607
:100D3D00C2B1C287C281306002A143855056855130
:100D4D0057D26043E68022207D11C2AF754302C2A7
:100D5D0086D282D2AF759F02020F23C2AF754302B6
:100D6D00C286D280D2AF759F02020F23307243200C
:100D7D007D20C2AF754303900143757E40C281C291
:100D8D0080306204D287A197D286D2AF759F0302BD
:100D9D000F23C2AF754303900143757E40C2B1C2AC
:100DAD0082306204D287A1B7D286D2AF759F01027D
:100DBD000F23207D17C2AF75430390011EC28130F2
:100DCD006202D287D2AF759F03020F23C2AF754364
:100DDD000390011EC2B1306202D287D2AF759F015E
:100DED00020F23207D11C2AF754304C282D280D27F
:100DFD00AF759F01020F23C2AF754304C280D2822B
:100E0D00D2AF759F03020F23307243207D20C2AFF6
:100E1D00754305900132757E04C287C28630620427
:100E2D00D2B1C133D282D2AF759F02020F23C2AFAE
:100E3D00754305900154757E01C287C286306204E8
:100E4D00D281C153D280D2AF759F02020F23207D74
:100E5D0017C2AF754305900114C287306202D2B13B
:100E6D00D2AF759F02020F23C2AF754305900128C3
:100E7D00C2873062EBD281D2AF759F02020F232061
:100E8D007D11C2AF754306C280D286D2AF759F0366
:100E9D00020F23C2AF754306C282D286D2AF759FB1
:100EAD0001020F23307242207D20C2AF75430190A5
:100EBD000154757E01C2B1C282306204D281C1CFAC
:100ECD00D280D2AF759F01020F23C2AF754301903F
:100EDD000132757E04C281C280306204D2B1C1EF8D
:100EED00D282D2AF759F03E123207D16C2AF754329
:100EFD0001900128C2B1306202D281D2AF759F013B
:100F0D00E123C2AF754301900114C281306202D258
:100F1D00B1D2AF759F03C26622900112757E00C2D9
:100F2D00B1C287C281C282C286C280C2622278806B
:100F3D0076090876090876040876FF0876030876A0
:100F4D00FF087609087603087601087601788C7615
:100F5D00010876FF0876FF0876FF0876FF0876FF12
:100F6D000876030876FF0876FF0876FF08762508D1
:100F7D0076D00876280876500876040876FF08762D
:100F8D000208760008767A0876FF08760108760161
:100F9D00087600087603227887E6FFC272BF030247
:100FAD00D2727888E6C394036008C27DE630E10210
:100FBD00D27DC27E7889E630E102D27EC3EF940203
:100FCD006008758E01D273020FDC758E00C273221C
:100FDD007880E6149000809378A4F67881E61490DA
:100FED0000809378A5F67886E61490008D9378A608
:100FFD00F6789CE67538FF75390CB402067538A085
:10100D0075390AB4030675388275390578A3E61467
:10101D0090009A93F569120F2622C2B3789DE6606F
:10102D0002D2B3227896E6FA7897E6FB7888E6B492
:10103D000305C3EB940EFB307F047A007BFFC3EBFB
:10104D009AFCC3948250027C827575000575EC85FF
:10105D0075F0A4C3E5F0947D40F222D27F113112D8
:0F106D0005A77A007B007C1012059DE55F2AFA2B
:10107C0074003BFBDCF37C04C3EB13FBEA13FADCDC
:10108C00F7FEC27F113122E5EF20E6037520000543
:10109C0020903DFFE520146006901FFF1460009324
:1010AC0004600375EF1253D9BF7581C043FF8012E2
:1010BC00059875EF0243B203E5B3240420E70DF560
:1010CC0021E5B120E0068521B343B101120F26754D
:1010DC00803875A4C775F1FF75D4DF7590FF75A5C1
:1010EC000075F20075D50075A0FF75A60075F300AC
:1010FC0075D60075B0E475A71B75F4FF75E241E475
:10110C00F8F6D8FD756B01120F3B1215D178988645
:10111C0076753001C2AF1205B11205C11205A712C6
:10112C0005C81205A71205CF1205A7C2AF78FA7928
:10113C00FA308507D9FBD8F7021C00120FA4120F46
:10114C00DD1127113178988676120F267588507527
:10115C00891275C82475910475D84075A82275B884
:10116C000275E690759B80759D0075D10E75BC5807
:10117C0075BB0675BA1F75E880120598D2AF1208B8
:10118C00A553DACF207E0343DA20307E0343DA10F6
:10119C0043DA01C2D8C2711205B1D2617B037A0C59
:1011AC00E55E70077A0CDB030211371205A720707D
:1011BC0003021137C270E55FC3940240E1E52F547E
:1011CC001F856160F561B560D5DAD5C26153DACFA0
:1011DC00207E0343DA20307E0343DA10C2D8C2717A
:1011EC0078A2E67008D274E52F54E0F52FC275751D
:1011FC0029001205AC307409C3E529940A4002D2C7
:10120C007512059D78023074027800C3E55F984032
:10121C00F0C2AF1205C11205C11205C1D2AF120541
:10122C00B1754D007888E6B40302610E12059D7805
:10123C008CE6C39401500302130EE530C3940150A5
:10124C000302130E207435C3E55F94FF50030213A1
:10125C000EC2AF1205D6D2AF1205ACC3E55F940136
:10126C0050EFC2AF1205C11205A21205C1D2AF12C6
:10127C0005ACC3E55F94FF40E90217797F02D27F8A
:10128C0011311205ACC2AFC27F1131AE5FC3E55F45
:10129C00947FD2AF4076120598C2AF1205D6D2AF6A
:1012AC00DFDC1168C3EE94057897F61205B11216BF
:1012BC00131216FC7F0AD27F11311205ACC2AFC2D9
:1012CC007F1131AE5FC3E55F947FD2AF50E612055C
:1012DC0098C2AF1205C11205A21205C1D2AFDFD65A
:1012EC001168EE24057896F61205B1121613121732
:1012FC002B1205AC1131C3E55F94FF500241500233
:10130C001779C3E55F954D4003855F4D1205AC78A9
:10131C00017988E7B403027805C3E55F9840024180
:10132C0030C2AF1205D61205D61205D6D2AF1205B1
:10133C00B1753000E4F531F5320531E531F4703931
:10134C000532789AE67819146012783214600D78A8
:10135C007D14600878FA146003753200C3E5329886
:10136C00401715327531B478998676C2AF1205D60E
:10137C00D2AF789886761205AC1205A2E52A7005D4
:10138C00307402213778012074027806C3E55F9827
:10139C0040A77888E6C3940360031205ACE52A7075
:1013AC0003021137C2AF120F26E4F522F523F52400
:1013BC00F525F526F56AD2AF7885E6C333F568E4F2
:1013CC00F545F546F547F548F549F573F52CF52D3A
:1013DC00F53775730875BB1E1205981208A9E5E858
:1013EC0020ECFBA8BDA9BEE97001F888741208AD09
:1013FC0075730875BB1E7887E6FE7602120FA4780B
:10140C0087EEF6C2AF7564FF12094585226485220A
:10141C0065852266D2AF752201752401752501758B
:10142C00260185636C756D017888E6B40307C27D6F
:10143C00307602D27DD268D269753300120E8C12CE
:10144C000EB112096512096C12096512096C1209A8
:10145C006502146DC2AF120FA4D2AF75730075BBC9
:0D146C0006120BF01206A1120D0A120D540B
:1014790012096C120BDF306D031206FD206703128F
:10148900084830670312088F120D0A120D791209E4
:101499006C120BF0306D03120732120D0A120DF0A7
:1014A90012096C120BDF306D03120790120D0A122C
:1014B9000E1512096C120BF0306D031207ED120DA7
:1014C9000A120E8C12096C1208A9120BDF120D0AEE
:1014D900120EB11208AD12096C306935206B3285D4
:1014E900676485676585636C756D0179187A0CC3C6
:1014F900E53399400FC269D26A8A35856764856781
:101509006602151AC3E55F9401400302146D0215C2
:1015190097306A1B206B18E535147004C26A816024
:10152900F535C3E55F9401400302146D0215977503
:101539003600C3E56278FA985054307404E52A609D
:101549004D7888E6B40317207D05207607A167301A
:101559007602A167206B07D26B85676481AC78F04E
:10156900306B058567647820C3E541985002816D29
:10157900306B1BC26BC27D307602D27DD26A753563
:1015890012856764816D0536E55F6002A19A75363B
:1015990000C2AF120F267887E6FE7602120FA478F2
:1015A90087EEF6E4F522F523F524F525F526F56809
:1015B900C268D2AF120598120F26307409C3E536F6
:1015C9009405400221376140901A0D782012165572
:1015D900E520B4550CA3121655E520B4AA0302154B
:1015E900F3120F3B121613021612901A0378807B1E
:1015F9000A121655A308DBF9901A0F788C7B18127A
:101609001655A308DBF9901A2722C2AF12169412B5
:10161900166E901A00740E12165AA3740412165AF2
:10162900A3741412165A901A0378807B0A12165959
:10163900A308DBF9901A0F788C7B18121659A308A6
:10164900DBF91216A7121685901A2722E493F622BF
:10165900E6438F01538FFD75EF0275B7A575B7F195
:10166900F0538FFE22438F02438F0175EF0275B746
:10167900A575B7F1901A0DF0538FFC22901A0D74CD
:1016890055D15A901A0E74AAD15A227A3079D07843
:1016990020901A40D155E520F709A3DAF7227A30CC
:1016A90079D0901A40E7D15A09A3DAF922AB77A881
:1016B90078BB01027980BB02027981BB030279827E
:1016C900BB04027984BB05027986BB06027992BB09
:1016D90007027987BB080279A3BB0902799CBB0A77
:1016E900027988BB0B027989E8F7227C051205B1DA
:1016F900DCFB22C2AF1205C11205C81205CF1205C3
:10170900D61205A21205C11205C81205CF1205D6B7
:101719001205A21205C11205C81205CF1205D6D2AB
:10172900AF22C2AF1205D61205CF1205C81205C1E4
:101739001205A21205D61205CF1205C81205C1124B
:1017490005A21205D61205CF1205C81205C1D2AFDE
:1017590022AE77AF78C2AF1205C11205C11205C119
:101769001205A2DEF21205D61205A2DFF8D2AF22C7
:10177900D1FCD1F4D1F4757701757801757900F14F
:101789005A7C05AD5F1205B1C3ED955F70F5C3E5F0
:101799005F9401400AC3E55F94FF40320217B5D157
:1017A900B6D113D1FCC2AF75EF12D1F4DCD50579EE
:1017B900C3E5799403500280C6D1F40578E577141E
:1017C90090009F93F808C3E57898500280AED1F451
:1017D900D1F40577C3E577940C5002809C120F3B36
:0917E900D113C2AF75EF12D1F467
:0319FD0002109342
:101A00000E0414090904FF03FF0903010155AA018B
:101A1000FFFFFFFFFF03FFFFFF25D0285004FF0259
:081A2000007AFF01010003FF41
:101A4000235475726E6967794145343541232020EE
:101A500023424C48454C4923463331302320202033
:101A60002020202020202020202020202020202076
:101C0000C2AFC2D353D9BF7581C043B20343FF8073
:101C1000752438752503B1C975EF0275E24043F1AB
:101C20002053A4DF75D400D2857DFA780379E67C51
:101C300010752200752300901DD67B0675249875BB
:101C400025013085028142208508D8FBD9F9DCF7CF
:101C500081B4308508D8FBD9F9DCF781B4B189E4C7
:101C600093A3C39A6004DDC381B4DBDBB17B600264
:101C7000812B7B08E493FAA3B15CDBF87A30B15C8A
:101C8000752200752300B17BEAFCEBFDC3ED94FEE9
:101C9000400EB17B8A278B28ED30E0048A828B834B
:101CA000B17B7AC270D8C3ED94FE601350CEBD00F4
:101CB00025EC60097520007521FF0200008100A855
:101CC00027A9280809D804D90281D3B17FEA89AAB3
:101CD000F281C50D81A0C3ED94035049EDA2E092BD
:101CE000007AC5C3E5829400E583941C50902000DF
:101CF00010438F02438F0175B7A575B7F1F030001F
:101D00001FA827A9280809438F01538FFDD804D99C
:101D100002A12089AAE275B7A575B7F1F0A3A10DBC
:101D2000538FFC817C7AC1BD030CE493A3FAB140CC
:101D3000DCF8B138817C817EAA22AB23B15CEBFA5E
:101D4000EA6222752608C3E52313F523E52213F57D
:101D50002250066323A0632201D526EAB1C9B1C986
:101D600075260AEAF4200102D285300102C285B14B
:101D7000C9C3134002C201D526EB22B17FEAFB2082
:101D80008502A17F308502A184752608AE24AF2587
:101D9000C3EF13FFEE13FEB1CDB1C9C3EA13308513
:101DA000024480FA30E703632201C3E52313F523DD
:101DB000E52213F52250066323A0632201D526D91C
:101DC000E52265236523F52222AE24AF250E0FDE22
:101DD000FEDFFCD20122424C48656C693437316326
:041DE000F3100601F5
:00000001FF
